 rtl8169

 Timestamp is 3f4c91cc (Wed Aug 27 19:11:08 2003)

 Preferred load address is 10000000

 Start         Length     Name                   Class
 0001:00000000 00000469H .rdata                  CODE
 0001:0000046c 0000004cH .rdata$debug            CODE
 0001:000004b8 00007b9eH .text                   CODE
 0001:00008058 00000028H .idata$2                CODE
 0001:00008080 00000014H .idata$3                CODE
 0001:00008094 000000f8H .idata$4                CODE
 0001:0000818c 00000594H .idata$6                CODE
 0001:00008720 0000004aH .edata                  CODE
 0002:00000000 000000f8H .idata$5                DATA
 0002:000000f8 00000004H .CRT$XCA                DATA
 0002:000000fc 00000004H .CRT$XCZ                DATA
 0002:00000100 00000004H .CRT$XIA                DATA
 0002:00000104 00000004H .CRT$XIZ                DATA
 0002:00000108 00000004H .CRT$XPA                DATA
 0002:0000010c 00000004H .CRT$XPZ                DATA
 0002:00000110 00000004H .CRT$XTA                DATA
 0002:00000114 00000004H .CRT$XTZ                DATA
 0002:00000118 00000768H .data                   DATA
 0002:00000880 00000010H .bss                    DATA

  Address         Publics by Value              Rva+Base     Lib:Object

 0001:0000001c       ??_C@_0CC@DKEM@xxx?5RTL8169?5Initialize?5Failed?5xx@ 1000101c     gig_main.obj
 0001:00000040       ??_C@_0CI@KBAE@ooo?5RTL8169?5Initialize?5Successfu@ 10001040     gig_main.obj
 0001:00000068       ??_C@_1BC@FPJN@?$AAR?$AAT?$AAL?$AAL?$AAA?$AAN?$AAI?$AAC?$AA?$AA@ 10001068     gig_init.obj
 0001:0000007c       ??_C@_1BE@HOJK@?$AAM?$AAW?$AAI?$AAE?$AAn?$AAa?$AAb?$AAl?$AAe?$AA?$AA@ 1000107c     gig_init.obj
 0001:00000090       ??_C@_19CBLD@?$AAM?$AAC?$AAW?$AAA?$AA?$AA@ 10001090     gig_init.obj
 0001:0000009c       ??_C@_1BE@OFKD@?$AAT?$AAh?$AAr?$AAe?$AAs?$AAh?$AAo?$AAl?$AAd?$AA?$AA@ 1000109c     gig_init.obj
 0001:000000b0       ??_C@_1BG@GBJD@?$AAD?$AAu?$AAp?$AAl?$AAe?$AAx?$AAM?$AAo?$AAd?$AAe?$AA?$AA@ 100010b0     gig_init.obj
 0001:000000c8       ??_C@_1BE@MNKM@?$AAL?$AAa?$AAr?$AAg?$AAe?$AAs?$AAe?$AAn?$AAd?$AA?$AA@ 100010c8     gig_init.obj
 0001:000000dc       ??_C@_1BG@DKD@?$AAC?$AAk?$AAs?$AAO?$AAf?$AAf?$AAl?$AAo?$AAa?$AAd?$AA?$AA@ 100010dc     gig_init.obj
 0001:000000f4       ??_C@_1BG@HHIE@?$AAJ?$AAu?$AAm?$AAb?$AAo?$AAf?$AAr?$AAa?$AAm?$AAe?$AA?$AA@ 100010f4     gig_init.obj
 0001:0000010c       ??_C@_1BK@LJEM@?$AAS?$AAu?$AAp?$AAp?$AAo?$AAr?$AAt?$AA8?$AA0?$AA2?$AA1?$AAp?$AA?$AA@ 1000110c     gig_init.obj
 0001:00000128       ??_C@_1BG@MOMC@?$AAR?$AAx?$AAD?$AAm?$AAa?$AAC?$AAo?$AAu?$AAn?$AAt?$AA?$AA@ 10001128     gig_init.obj
 0001:00000140       ??_C@_1BM@NIOA@?$AAT?$AAx?$AAM?$AAa?$AAx?$AAD?$AAM?$AAA?$AAB?$AAu?$AAr?$AAs?$AAt?$AA?$AA@ 10001140     gig_init.obj
 0001:0000015c       ??_C@_1CC@KJCF@?$AAE?$AAa?$AAr?$AAl?$AAy?$AAR?$AAx?$AAT?$AAh?$AAr?$AAe?$AAs?$AAh?$AAo?$AAl?$AAd?$AA?$AA@ 1000115c     gig_init.obj
 0001:00000180       ??_C@_1CC@OBPK@?$AAE?$AAa?$AAr?$AAl?$AAy?$AAT?$AAx?$AAT?$AAh?$AAr?$AAe?$AAs?$AAh?$AAo?$AAl?$AAd?$AA?$AA@ 10001180     gig_init.obj
 0001:000001a4       ??_C@_1BE@DPFB@?$AAC?$AAo?$AAn?$AAn?$AAe?$AAc?$AAt?$AAo?$AAr?$AA?$AA@ 100011a4     gig_init.obj
 0001:000001b8       ??_C@_1BO@BKCK@?$AAN?$AAe?$AAt?$AAw?$AAo?$AAr?$AAk?$AAA?$AAd?$AAd?$AAr?$AAe?$AAs?$AAs?$AA?$AA@ 100011b8     gig_init.obj
 0001:000001d8       ??_C@_1BI@IKAC@?$AAN?$AAu?$AAm?$AAC?$AAo?$AAa?$AAl?$AAe?$AAs?$AAc?$AAe?$AA?$AA@ 100011d8     gig_init.obj
 0001:000001f0       ??_C@_1BE@PNCA@?$AAN?$AAu?$AAm?$AAR?$AAx?$AAD?$AAe?$AAs?$AAc?$AA?$AA@ 100011f0     gig_init.obj
 0001:00000204       ??_C@_1BK@OHHK@?$AAN?$AAu?$AAm?$AAT?$AAx?$AAD?$AAe?$AAs?$AAc?$AAH?$AAP?$AAQ?$AA?$AA@ 10001204     gig_init.obj
 0001:00000220       ??_C@_1BE@BKEM@?$AAN?$AAu?$AAm?$AAT?$AAx?$AAD?$AAe?$AAs?$AAc?$AA?$AA@ 10001220     gig_init.obj
 0001:00000234       ??_C@_1BE@MGG@?$AAN?$AAu?$AAm?$AAT?$AAc?$AAb?$AAH?$AAP?$AAQ?$AA?$AA@ 10001234     gig_init.obj
 0001:00000248       ??_C@_1O@FHLN@?$AAN?$AAu?$AAm?$AAT?$AAc?$AAb?$AA?$AA@ 10001248     gig_init.obj
 0001:00000258       ??_C@_1O@HMAH@?$AAN?$AAu?$AAm?$AAR?$AAf?$AAd?$AA?$AA@ 10001258     gig_init.obj
 0001:00000268       ??_C@_0FB@PAKN@Realtek?5RTL8169?18110?5Family?5Giga@ 10001268     gig_req.obj
 0001:000002f0       ??_C@_0CE@HFHN@xxx?5RTL8139C?$CL?5Initialize?5Failed?5@ 100012f0     rtl_main.obj
 0001:00000314       ??_C@_0CI@MEMO@?$CK?$CK?5RTL8139C?$CL?5Initialize?5Successf@ 10001314     rtl_main.obj
 0001:0000033c       ??_C@_1BA@ELGJ@?$AAC?$AAo?$AAn?$AAg?$AAe?$AAs?$AAt?$AA?$AA@ 1000133c     rtl_init.obj
 0001:0000034c       ??_C@_1BI@NAIM@?$AAW?$AAa?$AAk?$AAe?$AAU?$AAp?$AAF?$AAr?$AAa?$AAm?$AAe?$AA?$AA@ 1000134c     rtl_init.obj
 0001:00000364       ??_C@_1O@CAMP@?$AAL?$AAi?$AAn?$AAk?$AAU?$AAp?$AA?$AA@ 10001364     rtl_init.obj
 0001:00000374       ??_C@_1BC@HJNK@?$AAW?$AAI?$AAN?$AA9?$AA8?$AAA?$AAP?$AAM?$AA?$AA@ 10001374     rtl_init.obj
 0001:00000388       ??_C@_1BG@LGJN@?$AAE?$AAn?$AAa?$AAb?$AAl?$AAe?$AAL?$AAD?$AAP?$AAS?$AA?$AA@ 10001388     rtl_init.obj
 0001:000003a0       ??_C@_1BA@MEPM@?$AAO?$AAf?$AAf?$AAl?$AAo?$AAa?$AAd?$AA?$AA@ 100013a0     rtl_init.obj
 0001:000003b0       ??_C@_1M@EBOO@?$AAT?$AAx?$AAI?$AAF?$AAG?$AA?$AA@ 100013b0     rtl_init.obj
 0001:000003bc       ??_C@_1BI@HPGG@?$AAR?$AAe?$AAc?$AAv?$AAT?$AAr?$AAa?$AAf?$AAf?$AAi?$AAc?$AA?$AA@ 100013bc     rtl_init.obj
 0001:000003d4       ??_C@_1BM@NHGP@?$AAR?$AAx?$AAM?$AAa?$AAx?$AAD?$AAM?$AAA?$AAB?$AAu?$AAr?$AAs?$AAt?$AA?$AA@ 100013d4     rtl_init.obj
 0001:000003f0       ??_C@_0CI@LPGA@?$CK?$CK?5REALTEK?3?5Interrupt?3?$CFd?5?5IOPAdd@ 100013f0     rtl_init.obj
 0001:00000418       ??_C@_0FB@NAOA@Realtek?5RTL8139c?$CL?5Fast?5Ethernet?5@ 10001418     rtl_req.obj
 0001:000004b8       _GigMPInitialize           100014b8 f   gig_main.obj
 0001:000006db       _GigCheckForHang           100016db f   gig_main.obj
 0001:0000075f       _GigReset                  1000175f f   gig_main.obj
 0001:00000956       _GigSendPackets            10001956 f   gig_main.obj
 0001:00000b74       _MP_GET_STATUS_FROM_FLAGS  10001b74 f i gig_main.obj
 0001:00000baa       _GigReturnPacket           10001baa f   gig_main.obj
 0001:00000c0e       _NICReadRegParameters69    10001c0e f   gig_init.obj
 0001:00000d3d       _NICReadAdapterInfo        10001d3d f   gig_init.obj
 0001:00000d3d       _NICReadAdapterInfo69      10001d3d f   gig_init.obj
 0001:00000d9d       _NICInitSend69             10001d9d f   gig_init.obj
 0001:00000e67       _NICInitRecv69             10001e67 f   gig_init.obj
 0001:00000fb0       _NICInitializeAdapter69    10001fb0 f   gig_init.obj
 0001:00001106       _HwConfigure69             10002106 f   gig_init.obj
 0001:0000116a       _MpFreeAdapter69           1000216a f   gig_init.obj
 0001:0000141f       _SetupTBILink              1000241f f   gig_link.obj
 0001:0000143e       _SetupSpeedDuplexMode      1000243e f   gig_link.obj
 0001:00001513       _WriteOurCapability69      10002513 f   gig_link.obj
 0001:00001596       _Setup2ndNway69            10002596 f   gig_link.obj
 0001:00001617       _RestartNway69             10002617 f   gig_link.obj
 0001:00001653       _LinkChangeReNwayTimer69   10002653 f   gig_link.obj
 0001:000016ab       _NwayCheckingTimer69       100026ab f   gig_link.obj
 0001:0000171d       _InitialNwayCheckingTimer69 1000271d f   gig_link.obj
 0001:00001780       _GIGLinkDetectionDpc       10002780 f   gig_link.obj
 0001:0000183a       _GIGProcessLinkChange      1000283a f   gig_link.obj
 0001:0000191a       _MP_WritePhyUshort         1000291a f   gig_link.obj
 0001:00001965       _MP_ReadPhyUshort          10002965 f   gig_link.obj
 0001:000019ae       _GigQueryInformation       100029ae f   gig_req.obj
 0001:00001def       _GigGetStatsCounters       10002def f   gig_req.obj
 0001:00001def       _NICGetStatsCounters       10002def f   gig_req.obj
 0001:00001f4d       _GigSetInformation         10002f4d f   gig_req.obj
 0001:000020f3       _GigSendPacket             100030f3 f   gig_nic.obj
 0001:000023bf       _NICSendPacket69           100033bf f   gig_nic.obj
 0001:0000254e       _NICStartSend69            1000354e f   gig_nic.obj
 0001:00002561       _RxStatistic69             10003561 f   gig_nic.obj
 0001:0000258e       _GigHandleRecvInterrupt    1000358e f   gig_nic.obj
 0001:000027b3       _ReuseRxDesc69             100037b3 f   gig_nic.obj
 0001:00002821       _GetRxDesc69               10003821 f   gig_nic.obj
 0001:000028be       _NICReturnRFD69            100038be f   gig_nic.obj
 0001:00002919       _NICResetRecv69            10003919 f   gig_nic.obj
 0001:00002a3d       _GigOnQueryTaskOffload     10003a3d f   offloadgig.obj
 0001:00002c59       _GigOnSetTaskOffload       10003c59 f   offloadgig.obj
 0001:00002eab       _QueryOffloadInfo69        10003eab f   offloadgig.obj
 0001:00002f34       _LargeSend_SetByteTransmitted69 10003f34 f   offloadgig.obj
 0001:00002f58       _NICRxVerifyChecksum69     10003f58 f   offloadgig.obj
 0001:00003016       _DriverEntry               10004016 f   rtl_main.obj
 0001:000030a9       _MPInitialize              100040a9 f   rtl_main.obj
 0001:00003370       _MPCheckForHang            10004370 f   rtl_main.obj
 0001:0000341e       _MPHalt                    1000441e f   rtl_main.obj
 0001:00003496       _MPReset                   10004496 f   rtl_main.obj
 0001:00003670       _MPReturnPacket            10004670 f   rtl_main.obj
 0001:00003708       _MPSendPackets             10004708 f   rtl_main.obj
 0001:0000393f       _MPShutdown                1000493f f   rtl_main.obj
 0001:0000399e       _MPIsr                     1000499e f   rtl_main.obj
 0001:000039f7       _MPHandleInterrupt         100049f7 f   rtl_main.obj
 0001:00003a33       _MpFindAdapter             10004a33 f   rtl_init.obj
 0001:00003b6e       _NICAllocAdapterMemory69   10004b6e f   rtl_init.obj
 0001:0000414c       _MpAllocAdapterBlock       1000514c f   rtl_init.obj
 0001:00004251       _MpFreeAdapter             10005251 f   rtl_init.obj
 0001:00004506       _NICReadRegParameters      10005506 f   rtl_init.obj
 0001:00004635       _NICAllocAdapterMemory     10005635 f   rtl_init.obj
 0001:00004b64       _NICInitSend               10005b64 f   rtl_init.obj
 0001:00004c3c       _NICInitRecv               10005c3c f   rtl_init.obj
 0001:00004d6d       _NICFreeRfd                10005d6d f   rtl_init.obj
 0001:00004dc5       _NICAllocRfd               10005dc5 f   rtl_init.obj
 0001:00004dc5       _NICAllocRfd69             10005dc5 f   rtl_init.obj
 0001:00004ea0       _NICFreeRfd69              10005ea0 f   rtl_init.obj
 0001:00004f08       _NICInitializeAdapter      10005f08 f   rtl_init.obj
 0001:0000504c       _HwSoftwareReset           1000604c f   rtl_init.obj
 0001:00005070       _HwConfigure               10006070 f   rtl_init.obj
 0001:00005166       _HwSetupIAAddress          10006166 f   rtl_init.obj
 0001:000051ba       _HwClearAllCounters        100061ba f   rtl_init.obj
 0001:0000522f       _MPQueryInformation        1000622f f   rtl_req.obj
 0001:00005559       _ComputeCrc                10006559 f   rtl_req.obj
 0001:000055a2       _GetMulticastBit           100065a2 f   rtl_req.obj
 0001:000055cd       _NICSetMulticastList       100065cd f   rtl_req.obj
 0001:00005672       _NICSetPacketFilter        10006672 f   rtl_req.obj
 0001:00005703       _MPSetInformation          10006703 f   rtl_req.obj
 0001:000058c5       _MpFreeQueuedSendPackets   100068c5 f   rtl_nic.obj
 0001:00005924       _MpFreeBusySendPackets     10006924 f   rtl_nic.obj
 0001:00005980       _MP_FREE_SEND_PACKET       10006980 f i rtl_nic.obj
 0001:00005a94       _GMP_FREE_SEND_PACKET      10006a94 f i rtl_nic.obj
 0001:00005bab       _MpSendPacket              10006bab f   rtl_nic.obj
 0001:00005ea2       _MpCopyPacket              10006ea2 f   rtl_nic.obj
 0001:00005f3e       _MpStartPacketPhysicalMapping 10006f3e f   rtl_nic.obj
 0001:00005fee       _NICSendPacket             10006fee f   rtl_nic.obj
 0001:00006159       _NICStartSend              10007159 f   rtl_nic.obj
 0001:0000616f       _TxStatistic               1000716f f   rtl_nic.obj
 0001:0000618e       _MpHandleSendInterrupt     1000718e f   rtl_nic.obj
 0001:000063bb       _NextTxDesc                100073bb f   rtl_nic.obj
 0001:000063d8       _NextTxDescHPQ             100073d8 f   rtl_nic.obj
 0001:000063f5       _GetTxDesc                 100073f5 f   rtl_nic.obj
 0001:00006444       _GetTxDescHPQ              10007444 f   rtl_nic.obj
 0001:00006493       _RxStatistic               10007493 f   rtl_nic.obj
 0001:000064c0       _MpHandleRecvInterrupt     100074c0 f   rtl_nic.obj
 0001:000066ea       _ReuseRxDesc               100076ea f   rtl_nic.obj
 0001:00006758       _GetRxDesc                 10007758 f   rtl_nic.obj
 0001:000067e0       _NICReturnRFD              100077e0 f   rtl_nic.obj
 0001:0000683b       _NICStartRecv              1000783b f   rtl_nic.obj
 0001:0000683b       _NICSelfTest               1000783b f   rtl_nic.obj
 0001:0000683e       _NICResetRecv              1000783e f   rtl_nic.obj
 0001:00006962       _DumpTallyCounter          10007962 f   rtl_nic.obj
 0001:00006a84       _MpLinkDetectionDpc        10007a84 f   rtl_nic.obj
 0001:00006b3a       _NICOnQueryTaskOffloadcp   10007b3a f   offloadcp.obj
 0001:00006d26       _NICOnSetTaskOffloadcp     10007d26 f   offloadcp.obj
 0001:00006e9f       _QueryOffloadInfo          10007e9f f   offloadcp.obj
 0001:00006ee7       _LargeSend_SetByteTransmitted 10007ee7 f   offloadcp.obj
 0001:00006f0b       _NICRxVerifyChecksum       10007f0b f   offloadcp.obj
 0001:00006f96       _VerifySegment             10007f96 f   offloadcp.obj
 0001:00007056       _NICEnableInterrupt        10008056 f   routines.obj
 0001:00007081       _NICDisableInterrupt       10008081 f   routines.obj
 0001:0000709b       _ClearConfigBit            1000809b f   routines.obj
 0001:000070cf       _SetConfigBit              100080cf f   routines.obj
 0001:000070fd       _ExAllocateFromNPagedLookasideList 100080fd f   routines.obj
 0001:0000711a       _ExDeleteNPagedLookasideList 1000811a f   routines.obj
 0001:0000711b       _MpHandleCollision         1000811b f   intcp.obj
 0001:0000729b       _ReArrangeNumRxDesc        1000829b f   intcp.obj
 0001:000072e2       _PriorityPacket            100082e2 f   intcp.obj
 0001:000072fd       _PerPacketPriority         100082fd f   intcp.obj
 0001:0000730b       _ShortDesc                 1000830b f   intcp.obj
 0001:0000732d       _HandleRecvPriorityPacket69 1000832d f   intcp.obj
 0001:0000732d       _HandleRecvPriorityPacket  1000832d f   intcp.obj
 0001:00007350       _NICSendHPQPacket          10008350 f   intcp.obj
 0001:000074cd       _NICStartSendHPQ           100084cd f   intcp.obj
 0001:000074e3       _NICStartSendHPQ69         100084e3 f   intcp.obj
 0001:000074f6       _NICSetPCIBusEfficiency    100084f6 f   intcp.obj
 0001:00007887       _GigSavePhyPower           10008887 f   intcp.obj
 0001:00007a74       _AdjustRegParameters       10008a74 f   intcp.obj
 0001:00007af4       _SetupLink                 10008af4 f   link.obj
 0001:00007b97       _Setup2ndNway              10008b97 f   link.obj
 0001:00007c1e       _ProcessLinkChange         10008c1e f   link.obj
 0001:00007cc1       _WriteOurCapability        10008cc1 f   link.obj
 0001:00007d1e       _InitialNwayCheckingTimerProc 10008d1e f   link.obj
 0001:00007d81       _NwayCheckingTimerProc     10008d81 f   link.obj
 0001:00007e08       _RestartNway               10008e08 f   link.obj
 0001:00007e44       _LinkChangeReNwayTimerProc 10008e44 f   link.obj
 0001:00007ea5       _SetLDPS                   10008ea5 f   link.obj
 0001:00007eda       _DbgPrint                  10008eda f   ndis:NDIS.dll
 0001:00007ee0       _NdisStallExecution        10008ee0 f   ndis:NDIS.dll
 0001:00007ee6       _NdisFlushBuffer           10008ee6 f   ndis:NDIS.dll
 0001:00007eec       _NdisAdjustBufferLength    10008eec f   ndis:NDIS.dll
 0001:00007ef2       __allrem                   10008ef2 f   coredll:COREDLL.dll
 0001:00007ef8       __DllMainCRTStartup        10008ef8 f   corelibc:pegdmain.obj
 0001:00007f67       __cinit                    10008f67 f   corelibc:crt0dat.obj
 0001:0000802b       __cexit                    1000902b f   corelibc:crt0dat.obj
 0001:0000803a       _DllMain                   1000903a f   corelibc:dllmain.obj
 0001:00008050       _LocalFree                 10009050 f   coredll:COREDLL.dll
 0001:00008058       __IMPORT_DESCRIPTOR_NDIS   10009058     ndis:NDIS.dll
 0001:0000806c       __IMPORT_DESCRIPTOR_COREDLL 1000906c     coredll:COREDLL.dll
 0001:00008080       __NULL_IMPORT_DESCRIPTOR   10009080     ndis:NDIS.dll
 0002:00000000       __imp__DisableThreadLibraryCalls 1000a000     coredll:COREDLL.dll
 0002:00000004       __imp___allrem             1000a004     coredll:COREDLL.dll
 0002:00000008       __imp__LocalFree           1000a008     coredll:COREDLL.dll
 0002:0000000c       \177COREDLL_NULL_THUNK_DATA 1000a00c     coredll:COREDLL.dll
 0002:00000010       __imp__NdisMMapIoSpace     1000a010     ndis:NDIS.dll
 0002:00000014       __imp__NdisMRegisterIoPortRange 1000a014     ndis:NDIS.dll
 0002:00000018       __imp__NdisMSetAttributesEx 1000a018     ndis:NDIS.dll
 0002:0000001c       __imp__NdisReleaseSpinLock 1000a01c     ndis:NDIS.dll
 0002:00000020       __imp__NdisAcquireSpinLock 1000a020     ndis:NDIS.dll
 0002:00000024       __imp__NdisStallExecution  1000a024     ndis:NDIS.dll
 0002:00000028       __imp__NDIS_BUFFER_TO_SPAN_PAGES 1000a028     ndis:NDIS.dll
 0002:0000002c       __imp__NdisQueryBufferOffset 1000a02c     ndis:NDIS.dll
 0002:00000030       __imp__NdisCloseConfiguration 1000a030     ndis:NDIS.dll
 0002:00000034       __imp__NdisReadNetworkAddress 1000a034     ndis:NDIS.dll
 0002:00000038       __imp__NdisReadConfiguration 1000a038     ndis:NDIS.dll
 0002:0000003c       __imp__NdisOpenConfiguration 1000a03c     ndis:NDIS.dll
 0002:00000040       __imp__NdisMQueryAdapterResources 1000a040     ndis:NDIS.dll
 0002:00000044       __imp__NdisWritePciSlotInformation 1000a044     ndis:NDIS.dll
 0002:00000048       __imp__NdisMAllocateSharedMemory 1000a048     ndis:NDIS.dll
 0002:0000004c       __imp__NdisFreeSpinLock    1000a04c     ndis:NDIS.dll
 0002:00000050       __imp__NdisMFreeMapRegisters 1000a050     ndis:NDIS.dll
 0002:00000054       __imp__NdisFreeMemory      1000a054     ndis:NDIS.dll
 0002:00000058       __imp__NdisFreeBuffer      1000a058     ndis:NDIS.dll
 0002:0000005c       __imp__NdisMFreeSharedMemory 1000a05c     ndis:NDIS.dll
 0002:00000060       __imp__NdisFreePacketPool  1000a060     ndis:NDIS.dll
 0002:00000064       __imp__NdisFreeBufferPool  1000a064     ndis:NDIS.dll
 0002:00000068       __imp__NdisMDeregisterIoPortRange 1000a068     ndis:NDIS.dll
 0002:0000006c       __imp__NdisMUnmapIoSpace   1000a06c     ndis:NDIS.dll
 0002:00000070       __imp__NdisMDeregisterInterrupt 1000a070     ndis:NDIS.dll
 0002:00000074       __imp__NdisMInitializeTimer 1000a074     ndis:NDIS.dll
 0002:00000078       __imp__NdisMRegisterInterrupt 1000a078     ndis:NDIS.dll
 0002:0000007c       __imp__NdisDprReleaseSpinLock 1000a07c     ndis:NDIS.dll
 0002:00000080       __imp__NdisDprAcquireSpinLock 1000a080     ndis:NDIS.dll
 0002:00000084       __imp__NdisInterlockedIncrement 1000a084     ndis:NDIS.dll
 0002:00000088       __imp__NdisFlushBuffer     1000a088     ndis:NDIS.dll
 0002:0000008c       __imp__NdisAdjustBufferLength 1000a08c     ndis:NDIS.dll
 0002:00000090       __imp__NdisMRegisterMiniport 1000a090     ndis:NDIS.dll
 0002:00000094       __imp__NdisInitializeWrapper 1000a094     ndis:NDIS.dll
 0002:00000098       __imp__NdisInterlockedDecrement 1000a098     ndis:NDIS.dll
 0002:0000009c       __imp__NdisMCancelTimer    1000a09c     ndis:NDIS.dll
 0002:000000a0       __imp__NdisMDeregisterAdapterShutdownHandler 1000a0a0     ndis:NDIS.dll
 0002:000000a4       __imp__NdisSetEvent        1000a0a4     ndis:NDIS.dll
 0002:000000a8       __imp__NdisAllocateMemory  1000a0a8     ndis:NDIS.dll
 0002:000000ac       __imp__NdisAllocatePacketPoolEx 1000a0ac     ndis:NDIS.dll
 0002:000000b0       __imp__NdisAllocateBuffer  1000a0b0     ndis:NDIS.dll
 0002:000000b4       __imp__NdisAllocateBufferPool 1000a0b4     ndis:NDIS.dll
 0002:000000b8       __imp__NdisAllocateMemoryWithTag 1000a0b8     ndis:NDIS.dll
 0002:000000bc       __imp__NdisMAllocateMapRegisters 1000a0bc     ndis:NDIS.dll
 0002:000000c0       __imp__NdisSystemProcessorCount 1000a0c0     ndis:NDIS.dll
 0002:000000c4       __imp__NdisAllocateSpinLock 1000a0c4     ndis:NDIS.dll
 0002:000000c8       __imp__NdisInitializeEvent 1000a0c8     ndis:NDIS.dll
 0002:000000cc       __imp__NdisFreePacket      1000a0cc     ndis:NDIS.dll
 0002:000000d0       __imp__NdisAllocatePacket  1000a0d0     ndis:NDIS.dll
 0002:000000d4       __imp__NdisMCompleteBufferPhysicalMapping 1000a0d4     ndis:NDIS.dll
 0002:000000d8       __imp__NdisQueryBuffer     1000a0d8     ndis:NDIS.dll
 0002:000000dc       __imp__NdisMStartBufferPhysicalMapping 1000a0dc     ndis:NDIS.dll
 0002:000000e0       __imp__NdisGetCurrentSystemTime 1000a0e0     ndis:NDIS.dll
 0002:000000e4       __imp__NdisMRegisterAdapterShutdownHandler 1000a0e4     ndis:NDIS.dll
 0002:000000e8       __imp__DbgPrint            1000a0e8     ndis:NDIS.dll
 0002:000000ec       __imp__NdisSetTimer        1000a0ec     ndis:NDIS.dll
 0002:000000f0       __imp__NdisWriteErrorLogEntry 1000a0f0     ndis:NDIS.dll
 0002:000000f4       \177NDIS_NULL_THUNK_DATA   1000a0f4     ndis:NDIS.dll
 0002:000000f8       ___xc_a                    1000a0f8     corelibc:crt0init.obj
 0002:000000fc       ___xc_z                    1000a0fc     corelibc:crt0init.obj
 0002:00000100       ___xi_a                    1000a100     corelibc:crt0init.obj
 0002:00000104       ___xi_z                    1000a104     corelibc:crt0init.obj
 0002:00000108       ___xp_a                    1000a108     corelibc:crt0init.obj
 0002:0000010c       ___xp_z                    1000a10c     corelibc:crt0init.obj
 0002:00000110       ___xt_a                    1000a110     corelibc:crt0init.obj
 0002:00000114       ___xt_z                    1000a114     corelibc:crt0init.obj
 0002:00000118       _NICRegTable69             1000a118     gig_init.obj
 0002:000003d8       _GigSupportedOids          1000a3d8     gig_req.obj
 0002:00000488       _HighestAcceptableMax      1000a488     rtl_init.obj
 0002:00000490       _NICRegTable               1000a490     rtl_init.obj
 0002:000007d0       _NICSupportedOids          1000a7d0     rtl_req.obj
 0002:00000880       __exitflag                 1000a880     <common>
 0002:00000884       ___onexitend               1000a884     <common>
 0002:00000888       ___onexitbegin             1000a888     <common>
 0002:0000088c       __pRawDllMain              1000a88c     <common>

 entry point at        0001:00007ef8

 Static symbols

 0001:00007f89       __initterm                 10008f89 f   corelibc:crt0dat.obj
 0001:00007fa3       _doexit                    10008fa3 f   corelibc:crt0dat.obj
